:100A0600FFFEFCF8F0E0C0800080C0E0F0F8FCFEDD
:100A1600003F065B4F666D7D077F6FFEFDFBF7EFC0
:010A2600DFF0
:100A440002080096020A009602100000020E00003E
:080A5400020C0000C180C10189
:100A2700758911E4F58A758CDCC28DD28CD2A9D276
:0D0A3700AFF58B758DDCC28FD28ED2AB2255
:03000B00020800E8
:10080000C0E0C0F0C083C082C0D075D000C000C0BE
:1008100001C002C003C004C005C006C007758A003D
:10082000758CDCC28DE509150970021508E50945CE
:1008300008705274212511F582740A3510F583E48D
:1008400093FF120A5D7417250FF582740A350EF5B1
:1008500083E493FF120A74E5112401FFE43510FECE
:100860007C007D0612092C8C108D11E50F2401FFF0
:10087000E4350EFE7C007D0A12092C8C0E8D0F755E
:100880000800750996D007D006D005D004D003D053
:1008900002D001D000D0D0D082D083D0F0D0E032CE
:03001B000209B720
:1009B700C0E0C083C082C0D0758B00758DDCC28F4C
:1009C700E50B150B7002150AE50B450A7028F50CA7
:1009D700F50D7406250DF582740A350CF583E4933D
:1009E700F590050DE50D7002050C6410450C70E2DD
:0F09F700750A00750B96D0D0D082D083D0E03235
:100A5D00E4FDFCC2A78F80D2A70DBD00010CED6493
:060A6D00784C70F5C2A7F1
:010A73002260
:100A7400E4FDFCC2A68F80D2A60DBD00010CED647E
:060A8400784C70F5C2A6DB
:010A8A002249
:030000000208A053
:0C08A000787FE4F6D8FD7581200208E79F
:10092C00C2D5EC30E709B2D5E4C39DFDE49CFCEEE6
:10093C0030E715B2D5E4C39FFFE49EFE120962C3F3
:10094C00E49DFDE49CFC800312096230D507C3E4EE
:06095C009FFFE49EFE2255
:1008AC00020A27E493A3F8E493A34003F68001F231
:1008BC0008DFF48029E493A3F85407240CC8C3334D
:1008CC00C4540F4420C8834004F456800146F6DF1C
:1008DC00E4800B0102040810204080900A44E47E5E
:1008EC00019360BCA3FF543F30E509541FFEE49311
:1008FC00A360010ECF54C025E060A840B8E493A3D8
:10090C00FAE493A3F8E493A3C8C582C8CAC583CA02
:10091C00F0A3C8C582C8CAC583CADFE9DEE780BEBA
:010A5C000099
:10096200BC000BBE0029EF8DF084FFADF022E4CC79
:10097200F875F008EF2FFFEE33FEEC33FCEE9DEC42
:10098200984005FCEE9DFE0FD5F0E9E4CEFD22ED88
:10099200F8F5F0EE8420D21CFEADF075F008EF2FD2
:1009A200FFED33FD4007985006D5F0F222C398FDC3
:0509B2000FD5F0EA2260
:00000001FF
